:030000000208985B
:10089800758E3075D20078FFE4F6D8FD75819D021B
:0208A80008E561
:0F0EBE001209B7D2AED2BE120C34120A4180F420
:0405EF00029900006D
:020D6B00AD07D2
:100D6D00E4FCFBFAF527F52875FE2975FF8BEDC41C
:100D7D0054F04401F5A5E5A520E0FBAFA1AB07AF0D
:100D8D00A2EFFEEEFAEB2528F528EA3527F5270C1C
:100D9D00BC08DBE528AE277803CEC313CE13D8F9F4
:010DAD00FF46
:010DAE002222
:100DAF00E4F524F5257F05120D6B8E248F257F0624
:100DBF00120D6BE4FCFDC004A905AA06AB07AE2417
:100DCF00AF257C077DD0120271D0001201A98E24AD
:020DDF008F255E
:010DE10022EF
:100DE200E4F525F5267F04120D6B8E258F267F06EE
:100DF200120D6BE4FCFDC004A905AA06AB07AE25E3
:100E0200AF267C037DE8120271D0001201A98E2563
:020E12008F2629
:010E140022BB
:0605F300C114C116C11580
:10078900E4FFFE752401120DE2C3EF9474EE940E9A
:1007990040037F0122E5E630E757D3EF9436EE9424
:1007A900055030EF9422EE94024028301612EF944F
:1007B90014EE94055007C2167524018003E4F5244C
:1007C90030152ED3EF9444EE94024022C2157524BD
:1007D90001801ED3EF9436EE94054004D216800BA7
:1007E900C3EF9422EE94025002D21553B3FEE4F5FE
:0307F90024AF2406
:0107FC0022DA
:100BDF00E5E620E70953B3FE75F210C21422E5F2E1
:100BEF00540C601053B3FEE5F354C0603775F20C2C
:100BFF0075F3C022E5F354C0600375F3C012078983
:100C0F00EF6021E5F230E417C3789AE694EB18E62B
:100C1F00940F500575F210800353B3FED214224384
:050C2F00B301C2142214
:0405F900C117C1184D
:100D2500E5E530E103C21722E5E230E705C217D257
:100D35001822E5E830E00EC217300B29C20B75E822
:100D45000175B50122D21730181BE5E630E716C349
:100D5500789AE6941018E6940E4005D217C2182228
:060D6500E4F5B5C21722FF
:0705FD00011DFFC119C11A25
:100E4100E5E230E425E5E25408FF651D601CE5E2BA
:100E510030E305751C018005E4F51CC21ED219D2D0
:0A0E61001AE4F51FF540F5418F1D5E
:010E6B002264
:0B060400C113C111C110C112019D0003
:100E6C00301208C211C212789D7602301006C210E0
:0E0E7C00789D7603301306C213789D7601220E
:03060F000198004F
:10000E007893A607EDC31308F608A60508A603E421
:03001E0008F622BF
:100CD8007893E6603D24FE6007047036D283803442
:100CE8007897E6FFC37894965004D2838002C28333
:100CF800EFC3789596401DE47897F618E6FFF46000
:100D080013EFD394004001167896E670077893F6AF
:0D0D18008002C2837893E67898F6180622D0
:05061200011E00C11DE6
:100E9D00E5E620E706200903301D04C21DC322D359
:010EAD002222
:1009B700E4F5D275FE8943FF8075FE0153FFFCF510
:1009C700FE75FF0375FE0E75FF05D2DF4387807541
:1009D700BA0375AAFD7598D0D299D298D2AC75B7DB
:1009E700C3758901758CFC758A17D2A9D28C75FEDF
:1009F7000675FF0C75FE0375FF0CC283F58675FE41
:100A07000F43FF8075FE4F75FF1075FE1775FF3C8E
:100A170075FE1E75FF0CD2A8D2B9D2BBD2AF75F244
:100A27001C75F3C075E80C75FE8753FFDF43B310E1
:0A0A370075FE7043FF04751E0A22CD
:03000300020006F2
:0100060032C7
:03004B00020ED8CA
:060ED80075EB3CD21D3257
:03005B00020EDEB4
:060EDE0075F30CD21D3279
:0F0617000B880000000000000000000000C11C64
:100E8A0074882553F8A6990553E5532275520075BF
:030E9A00530022E0
:0A0E15008E358F368B378A38893905
:100E1F00E4FFEFC39536E495355016201BFD783768
:100E2F00E475F00112023B120154D21BF5990F80A9
:010E3F00E1D1
:010E4000228F
:0300230002092AA5
:0F092A00C0E0C0D075D000C000C005C006C00737
:10093900309904C299C21B309867C298E551146076
:100949001F04705DE599B4AA0F755101120E961234
:100959000E8A700205528049755100120E96804127
:10096900120E8A70020552640745527015788EE698
:10097900FEE42409FFE43EFE18E6FDEEF554EF4DD2
:10098900F555E55565537004E5546552600BD3E59B
:1009990053940BE55294004008120E96755100D2FB
:0109A9001C31
:0D09AA00D007D006D005D000D0D0D0E0326C
:05062600011F00C11ED0
:1006E000E5E630E729301402807A301A10E51CB4B0
:1006F000010B201E08D21EE4FBFDFF801D7898E64A
:1007000064027002E1887BFF7D647F028077301F86
:100710000F301A747B047D647F0212000EC21A220D
:10072000E51C6401704BE56B7004E56C6043E56BA0
:1007300064016005E56CB401167898E6640260090E
:100740007BFF7D327F0212000EE4F51FD21D22E5F1
:100750006B64027033E56C6402702DE51FC394284E
:100760005009051FE4FBFD7F01801AE4FBFDFF80BB
:1007700014E51FC394285009051FE4FBFD7F018089
:0907800004E4FBFDFF12000E224F
:100A4100300C08C20C120E41120D25300F05C20FD9
:100A5100120CD8300A1EC20A120E6C120BDF120DD4
:100A6100AF7899A60608A60712029E1206E0120B9D
:100A71001B120C89300D35C20DE51ED394004009BF
:100A8100151E301D27C21D8020120E9D501BC2ACA9
:100A9100C2BBC2B9C2A975FE2953FF7F438702D2E7
:0D0AA100ACD2BBD2B9D2A98000751E0A22CA
:0B004E000000000000000000000000A7
:10062B00C109C105C108C102C104C100C106014213
:10063B000002450000014400014300C101024700D4
:10064B0000027000000672000000000000087A0033
:10065B0000000000000000028400000256000002AF
:10066B00780000028600000282000002580000168B
:10067B005A00000000000000000000000000000015
:10068B0000000000000000013F00C1030240000019
:02069B00C10795
:10002600FF547FF6EFC4131313540122C208D20102
:10003600E4F544D20522FF5401F6EFC3135401221E
:100EAE00D282EF700753B7CF43B7302253B7CF225A
:10029E00E5E8540C60110542E542C394024008E4BF
:1002AE00F54275E80C8109301960301758200606A2
:1002BE0075B501D20622E4F56BF56CC205C200F5E8
:1002CE0045F546E51C7011D202C204C219D209C20C
:1002DE0006C28243B7308032C202C208C3E54194DF
:1002EE0002E5409400500FE4FF120EAE0541E541C9
:1002FE00701805408014E4F5B5D204C219C206F593
:10030E0040F54180057F01120EAE30042AC3E5414F
:10031E009458E5409402501AE54120E0047D248073
:10032E00027D257F0D12048F0541E54170090540C0
:10033E008005E4FF120EAE2002052000028184C368
:10034E00E5419432E54094005031E54120E00F3014
:10035E0000047D24800DE51C70187D24800F300074
:10036E00067D257F058008E51C70077D257F0D1213
:10037E00048F0541E541700205402230000DC20098
:10038E00C202C209E4F5B57F0181192002028184FF
:10039E00E5E354AC64AC6003301F12C3E5469458D9
:1003AE00E54594024007D200E4F540F54120072EC2
:1003BE00C3E5419464E5409400501AE54120E00401
:1003CE007D2480027D257F0E12048F0541E541704C
:1003DE000D05408009D207D208E4F540F5413008FA
:1003EE0050E544C3940150097D2412048508F6801B
:1003FE0030E543D394054006120032FF800D789409
:10040E00E6601208E66007120032FF020EAE7D258E
:10041E00120485800C7895E660077D247F0A12040D
:10042E008FE544D3941E40070543E4F5448002054E
:10043E00443005210541E54170020540D39414E591
:10044E004094004010C205E4F544F543D2827D216C
:10045E007F1202048F30011EE544C3946450097567
:10046E00FE7843FF03054422C201E4F54475FE788D
:10047E0053FFFC43FF01227F0A12048FE47894F6A7
:01048E00224B
:0A0AAE008B358A3689378C388D3974
:100AB800E4FDFC753A10753B21F53CE5391539AE76
:100AC80038700215384E60467835E475F001120228
:100AD8003B120154F53CFEEE6204E4F53DF53EC3DD
:100AE800E53E9408E53D940050D1EC30E70FED2544
:100AF800E0FFEC33653AFCE53B6FFD8007ED25E050
:100B0800FDEC33FC053EE53E70D5053D80D1AE04D5
:020B1800AF0527
:010B1A0022B8
:04048F008F248D2504
:1004930078267C007D007BFF7A00794E7E007F0BFF
:1004A30012012EE4F531F532F533F5347526AA85BC
:1004B3002527852428F529851C2AE52412024B05C6
:1004C3000C0504E10A05190B05200D054F0E058FD8
:1004D3000F051911059A120519370000059D752B93
:1004E3000EE4F52CFF74722FF8E6FE742D2FF8A698
:1004F300060FBF06F0E4FF747A2FF8E6FE74332F7D
:10050300F8A6060FBF08F0A19D752B01E4F52CA2F8
:100513000333F52DA19DE4F52BF52C807D752B057B
:10052300E4F52C752D10F52D752E01E5E654807834
:100533009C46F52FE525B4240478848007E525B48B
:1005430025057885E6F530E4F531804E752B0AE410
:10055300F52C853F2DFFEFFDE53F2DFDE433FCD367
:10056300ED9416EC648094804008742E2FF876FF87
:10057300800EE53F2F245AF8E6FE742E2FF8A606C8
:100583000FBF09D27409253FF53F800E752B01E497
:10059300F52C752D018003D20E22E52CFEE42407F1
:1005A300FFE43EF533EF452BF5347B007A007926E3
:1005B300FDAC33120AAE8E318F32AD3474272DF871
:1005C300A607E531FF74282DF8A607C28275FE0E33
:1005D30043FF04E534240AFFE43533FE7B007A004D
:0B05E3007926120E1575FE0E53FFF373
:0105EE0022EA
:100800007889E6C4540FFD540360020197EF24F683
:10081000602524FD602F14607124D7707AE4FE787F
:100820008DE6FFEEC39F506F748F2EF8E6FF747253
:100830002EF8A6070E80E8788FE6BD04047870F6DF
:10084000227871F622ED64047891701FE6788412A4
:1008500000267856F67892E6F54708E67878120092
:100860003C7886F67894E67882F622E6788512005F
:10087000267857F67892E6F54808E6787912003C33
:100880007887F67894E67883F622788FE6BD0404BC
:070890007858F6227859F6B2
:01089700223E
:100C8900E4F524F525F526301C44C21C788EE6FED1
:100C9900E42407FFE43EFE18E6FDEEF524EF4DF5EA
:100CA900257B007A007988FDAC24120AAEAC06AD2A
:100CB90007AB25748A2BF8E6FE74892BF8E6FBEB63
:0E0CC900B5050BEEB50407788AE6FF120800A9
:010CD70022FA
:10069D00019C00C11F019B1E14080BB80C1C0CE41F
:0E06AD000D480DAC0E420ED80F3C0FD2106857
:0B0ECD00EF25E02408F8E6FC08E62210
:100B1B00E4FFE5E630E715120ECD2432FDE43CFC94
:100B2B00C3789AE69D18E69C50108012120ECDFDEC
:100B3B00C3789AE69D18E69C40040FBF0AD4789CB4
:100B4B00E6FEEFD39E400418068003789B16789B35
:100B5B00E6FED394325006EEC3940A5007789CA657
:100B6B000718761E789CE6FFD394015003D21F2200
:080B7B00EFD394024002C21FF7
:010B8300224F
:1006BB00014B00014D00014A00014900014C00C1F2
:1006CB000CC10FC10BC10AC10D015000014E00C17D
:0406DB000E014F00BD
:100C3400E5506050E4F550054BE54BC39405400581
:100C4400E4F54BD20C054DE54DC3940A4005E4F59B
:100C54004DD20F0549E549C394644005E4F549D2F2
:100C64000A054AE54AC394FA401AE4F54AD20B0548
:100C74004CE54C9404400DE4F54CD20D0546E54694
:050C840070020545228D
:03000B00020B8461
:100B8400C0E0C0D074FC258CF58C7417258AF58AD6
:100B9400755001054EE54EC39405403A754E00303C
:100BA4000E34E54FD394045004C282801BE54F30C9
:100BB400E00BB40D04C282800FD282800BE54FB4E7
:100BC4000E04D2828002C282054FE54FC3941740BF
:0B0BD40005C20E754F00D0D0D0E032FB
:1008AA00020EBEE493A3F8E493A34003F68001F298
:1008BA0008DFF48029E493A3F85407240CC8C3334F
:1008CA00C4540F4420C8834004F456800146F6DF1E
:1008DA00E4800B01020408102040809005EFE47EBA
:1008EA00019360BCA3FF543F30E509541FFEE49313
:1008FA00A360010ECF54C025E060A840B8E493A3DA
:10090A00FAE493A3F8E493A3C8C582C8CAC583CA04
:10091A00F0A3C8C582C8CAC583CADFE9DEE780BEBC
:0106DF00001A
:10005E00E709F608DFFA8046E709F208DFFA803E84
:10006E0088828C83E709F0A3DFFA8032E309F60871
:10007E00DFFA8078E309F208DFFA807088828C83D9
:10008E00E309F0A3DFFA806489828A83E0A3F6088D
:10009E00DFFA805889828A83E0A3F208DFFA804C67
:1000AE0080D280FA80C680D4806980F2803380103E
:1000BE0080A680EA809A80A880DA80E280CA8033A7
:1000CE0089828A83ECFAE493A3C8C582C8CCC5831F
:1000DE00CCF0A3C8C582C8CCC583CCDFE9DEE780EF
:1000EE000D89828A83E493A3F608DFF9ECFAA9F06E
:1000FE00EDFB2289828A83ECFAE0A3C8C582C8CCC4
:10010E00C583CCF0A3C8C582C8CCC583CCDFEADEDC
:10011E00E880DB89828A83E493A3F208DFF980CC3E
:10012E0088F0EF60010E4E60C388F0ED2402B40437
:10013E000050B9F582EB2402B4040050AF232345DE
:06014E0082239000AE7355
:10015400BB010689828A83E0225002E722BBFE02A9
:09016400E32289828A83E49322DC
:10016D0075F008758200EF2FFFEE33FECD33CDCC49
:10017D0033CCC58233C5829BED9AEC99E5829840CC
:10018D000CF582EE9BFEED9AFDEC99FC0FD5F0D6A9
:10019D00E4CEFBE4CDFAE4CCF9A88222B800C1B9D3
:1001AD000059BA002DEC8BF084CFCECDFCE5F0CB11
:1001BD00F97818EF2FFFEE33FEED33FDEC33FCEB4A
:1001CD0033FB10D703994004EB99FB0FD8E5E4F905
:1001DD00FA227818EF2FFFEE33FEED33FDEC33FCF2
:1001ED00C933C910D7059BE99A4007EC9BFCE99AE6
:1001FD00F90FD8E0E4C9FAE4CCFB2275F010EF2F2B
:10020D00FFEE33FEED33FDCC33CCC833C810D7072A
:10021D009BEC9AE899400AED9BFDEC9AFCE899F865
:0E022D000FD5F0DAE4CDFBE4CCFAE4C8F922F8
:10023B00FAE6FB0808E6F925F0F618E6CA3AF622C4
:10024B00D083D082F8E4937012740193700DA3A342
:10025B0093F8740193F5828883E473740293686056
:06026B00EFA3A3A380DF56
:10027100EC8EF0A4CCC5F0CCCDF8EFA4CEC5F02D1A
:10028100FDE43CFCE8A42EC8C5F03DFDE43CFCEFD8
:0D029100A4FFE5F028FEE43DFDE43CFC2266
:00000001FF
